S02B00002F686F6D652F74696D652F646F632F636F646566696C652F656D62652F426C6F672F73746D33322FBD
S3150800000000000220BD090008B9090008B709000860
S31508000010B7090008B7090008B7090008000000007A
S31508000020000000000000000000000000B9090008F8
S31508000030B909000800000000B9090008C904000849
S31508000040B7090008B7090008B7090008B709000882
S31508000050B7090008B7090008B7090008B709000872
S31508000060B7090008B7090008B7090008B709000862
S31508000070B7090008B7090008B7090008B709000852
S31508000290B7090008B709000880B500AF41F6044061
S315080002A000F07CFB082300220121104800F02BF9FE
S315080002B00823002200210D4800F045F908210B48C3
S315080002C000F012F90A4B1B68094A43F4807313605D
S315080002D041F6024000F062FB4FF40053022200216F
S315080002E0044800F010F900BF80BD00BF0010025896
S315080002F0004802580008025880B500AF4FF4407015
S3150800030000F0CFFB00F02CF84FF47A7000F0BCF840
S31508000310FFF7C2FF4FF400510F4800F0E8F8034614
S31508000320002BF7D0142000F095F84FF400510A4836
S3150800033000F0DDF80346002B03D00821074800F03B
S31508000340D9F800BF4FF40051034800F0D0F803462F
S31508000350002BF7D1DEE700BF00080258001002584C
S3150800036080B58CB000AF3B462C220021184600F021
S3150800037091FC41F6074000F011FB41F6816000F060
S315080003800DFB022301220121304800F0BCF80223AC
S31508000390022200212D4800F0D6F80023FB6203E074
S315080003A000BFFB6A0133FB62FB6A132BF8D90221F3
S315080003B0264800F097F800233B7002237B70244BF5
S315080003C07B6005233B72C0237B8102233B73022398
S315080003D07B730223BB7320233B7481237B82022316
S315080003E03B7502237B750223BB7520233B7681234D
S315080003F07B8302233B7702237B770223BB77002389
S3150800040087F82030082387F82130042387F822301C
S31508000410042387F82330042387F82430042387F835
S315080004202530042387F82630012387F8273002234E
S3150800043087F82830002387F829303B46184600F00D
S3150800044063F900BF3037BD4680BD00BF001C0258A7
S3150800045040787D0180B485B000AF7860094B1B6891
S31508000460FB6001E030BF00BF064B1A68FB68D31A71
S315080004707A689A42F6D800BF00BF1437BD465DF8C1
S31508000480047B70472400002080B582B000AF7860F6
S31508000490042000F0E9FA002000F042FA02467B68E0
S315080004A0B2FBF3F3013B184600F0D8FA00F0F4FA71
S315080004B00F21FF2000F0FEFA00F0E0FA00F0E5FA5E
S315080004C000BF0837BD4680BD80B400AF044B1B682B
S315080004D00133034A136000BFBD465DF8047B7047CD
S315080004E02400002081617047090481617047006912
S315080004F008407047436901EA030221EA030141EA19
S315080005000241816170472DE9F04105680026C468FB
S315080005104FF0030E43FA06F7FF070DD577000EFADC
S3150800052007FC01FA07F802FA07F725EA0C0524EA98
S315080005300C0448EA05053C430136102EEAD105604D
S31508000540C460BDE8F081012941680CBF194399438D
S31508000550F0B5416000248168032643FA04F5ED07E7
S3150800056007D5650006FA05F702FA05F521EA070137
S3150800057029430134102CF0D18160F0BD2DE9F043F8
S3150800058091F800C0BCF1000F00F0A580012A26D022
S31508000590574B9E1F022A18BF1E46013A554D002387
S315080005A0B1F8028045F8323008F1FF3355F8324089
S315080005B02343D4B245F83230A700B0FBFCF34E48CB
S315080005C0FFB2B3FBF0FCACF1030001284B4808D896
S315080005D00423D0F82CE4BB404EEA03030DE0484E52
S315080005E0DBE7ACF1050EBEF1030F76D80823D0F889
S315080005F02C9403FA07FE4EEA0903C0F82C340CFBC8
S3150800060008F3B3F5D27F09D8DFF8F0C00220DCF88A
S315080006102CE4B84040EA0E00CCF82C0467000879B0
S3150800062004EB4404E4B2B0B155F832C000F1FF3E21
S315080006304CEA4E2CDFF8C4E045F832C04FF4803C53
S31508000640DEF82C840CFA04FCB3FBF0F04CEA080C38
S31508000650CEF82CC430804879B0B155F832C000F1D4
S31508000660FF3E4CEA0E4CDFF894E045F832C04FF4F2
S31508000670003CDEF82C840CFA04FCB3FBF0F04CEAE0
S31508000680080CCEF82CC47080897999B155F83200D7
S3150800069001F1FF3C40EA0C6045F832004FF4802235
S315080006A01648A240D0F82C54B3FBF1F32A43C0F8FD
S315080006B02C24B380114AFFB24FF08073D2F800148D
S315080006C0BB400B43C2F800344FF00073BB40D2F86E
S315080006D000141942FBD0BDE8F083DFF828E0734523
S315080006E08DD94FF00C0ED0F82C340EFA07FE73E7AE
S315080006F01A0000203044025840420F0000400258B9
S315080007000E0000203F548900F8B5814B0446D3F803
S31508000710002442F00102C3F80024D3F8102422F082
S315080007200702C3F81024D3F8102412F0380FFAD1B0
S315080007300122C3F8002494F8291094F8280000F040
S315080007402FFA94F8270000F057FA94F8260000F0DC
S31508000750D3F994F82630002B00F0C58000F0BCF9D8
S3150800076063688BB16A4BD3F8002442F48032C3F82D
S315080007700024D3F800249203FBD563684FF47A72F9
S31508000780B3FBF2F3634A1384237C227A1B03617852
S3150800079043EA0213227E0B4343EA02535C4AC2F839
S315080007A02834002900F0A2806568002304F10801B6
S315080007B02846C2F82C340122FFF7E0FE022204F193
S315080007C010012846FFF7DAFE2846032204F118012D
S315080007D0FFF7D4FE23784F48002B40F08980C38961
S315080007E094F8245000264A4F94F8201094F82120B3
S315080007F003800729C7F818644FEA0516D7F818C4FE
S3150800080046EA012646EA020646EA0C06C7F81864CE
S3150800081006D90B2994BF0739063943FA01F18BB279
S31508000820072A438009D90B2A95BF073A911F43FA2D
S3150800083002F20B4194BF93B29BB2032D94F8231096
S31508000840334E8CBFEA1E1A464FF00005838084BFDC
S3150800085043FA02F292B20329428194F82220C6F89A
S315080008601C544FEA01258CBF0339194645EA02157F
S31508000870D6F81C7488BF43FA01F145EA070588BF14
S3150800088089B2032AC6F81C548CBF033A1A4601815A
S3150800089088BF43FA02F294F8251088BF92B203295A
S315080008A0C2801B4AD2F820444FF00004C2F8204404
S315080008B0D2F8204444EA011484BF033943FA01F10B
S315080008C0C2F8204488BF8BB28381D2F8103443F033
S315080008D00303C2F81034D2F810340D4AC3F3C20326
S315080008E0032B0FD1F8BD00F0FFF839E70A4D5CE796
S315080008F0012B09BF63684023084AB3FBF2F308BF1C
S315080009009BB26DE7D2F81034C3F3C203E8E700BF21
S3150800091000400258000000200090D00340420F001B
S3150800092008B509282CD8DFE800F00A051C0A0D0DC1
S3150800093010131619154B1888154B584308BD134B39
S315080009405888F9E7114B9888F6E7104BD888F3E7EB
S315080009500E4B1889F0E70D4B5889EDE70B4B988934
S31508000960EAE70C4BD3F84C3413F0405FC3F301723B
S3150800097008D0022A08D1054B188C4FF47A73DCE7A5
S3150800098000F0A8F80448D9E70020D7E700000020BF
S3150800099040420F00004002580090D003430901224C
S315080009A000F01F0003F1B043824003F511331968C4
S315080009B00A431A607047FEE77047000038B51D4ABB
S315080009C01D4B1E498B4220D31D4A0021934221D339
S315080009D04FF0E0231B4C1C4DD3F8142D42F4007243
S315080009E0C3F8142DD3F8882D42F47002C3F8882D65
S315080009F0AC4212D3154C164DAC4212D3154CFFF728
S31508000A007BFC154DAC4210D338BD52F8040B43F8A5
S31508000A10040BD7E743F8041BD8E754F8043B984778
S31508000A20E6E754F8043B9847E6E754F8043B98474A
S31508000A30E8E700BF380D0008000000202400002069
S31508000A4028000020380D0008380D0008380D000869
S31508000A50380D0008380D0008380D000820F07F40D2
S31508000A604FF0E023586170474FF0E02200F0040091
S31508000A70136923F004030343136170474FF0E02220
S31508000A80136943F00203136170474FF0E0221369BC
S31508000A9043F00103136170474FF0E02300229A6187
S31508000AA0704740F0BF604FF0E02340F40030C3F8D1
S31508000AB00C0D7047952804D900F00F00044BC1545B
S31508000AC0704700F1604000F564400170704700BF50
S31508000AD014ED00E0FEE70000024A136843F4807351
S31508000AE01360704700200052024A136823F480738B
S31508000AF01360704700200052034A136823F00F035F
S31508000B0003431360704700BF00200052044AD2F81E
S31508000B100C3823F0070343F00203C2F80C38704779
S31508000B2000400258044AD2F80C3823F0070343F071
S31508000B300603C2F80C3870470040025808B50B0186
S31508000B4070B943F0040309485242D0F80C1802F071
S31508000B50020221F03F010A431A43C0F80C2808BDD7
S31508000B6009B9FFF7B7FF43F00C03ECE7004002585A
S31508000B70044AD2F80C3823F0070343F00103C2F8FD
S31508000B800C38704700400258044AD2F80C3823F053
S31508000B90070343F00503C2F80C38704700400258B3
S31508000BA008B5072807D8DFE800F0040C0F12121D55
S31508000BB01D21FFF7B7FF0F4AD2F804389B04FBD56F
S31508000BC008BDFFF7E1FFF6E7FFF7A0FFF3E7A0F19F
S31508000BD0040C0021DCF1000242EB0C020020FFF7B6
S31508000BE0ADFFE8E7053842424241F7E7FFF7C0FFA5
S31508000BF0E1E700BF00400258F8B5074608B9FFF715
S31508000C0069FF204B421E204E1B68C3F30B03B3F546
S31508000C10906F0FD1D6F818381C4923F440438A5CE4
S31508000C2043EA8233C6F81838174AD2F818389B04AC
S31508000C30FBD5F8BD1649B3F58A6FD6F818588C5CFB
S31508000C4025F440454FEA843418D141F68160FFF710
S31508000C50A5FE012F4FF0B0430AD145F44045C6F82A
S31508000C601858D3F82C2442F00102C3F82C24DBE7E9
S31508000C70D3F82C2422F00102C3F82C242C43C6F8FE
S31508000C801848D1E70010005C00400258340D0008EF
S31508000C90300D0008830730B546D08418844604E032
S31508000CA003F8011B9D0704D09C46A4456346F7D16B
S31508000CB030BD013A0244A2EB0C02032A29D9CCB270
S31508000CC004EB04240F2A04EB04442FD9A2F1100CD8
S31508000CD02CF00F0C03F11005AC44C3E90044C3E93A
S31508000CE0024410336345F8D112F00C0F02F00F0ED0
S31508000CF018D02EF0030C9C44AEF104051A4642F8AF
S31508000D00044B6245FBD125F0030404330EF00302BD
S31508000D102344002ACCD0C9B21A4403F8011B9342D3
S31508000D20FBD130BD7246F4E70346C6E79646E0E7D0
S30D08000D300003020103020100A1
S31508000D3840004000400040004000400040000000DD
S31508000D48000000000000000000000000000000008D
S30908000D580000000089
S705080009BD2C
